:10000000830100308A0004282030840043300F2010
:1000100083010A128A11AA2D04068001840A0406AB
:10002000031D0C28003483120313C300C41B2128B2
:10003000441B292844088A004308C30A0319C40A38
:1000400082008313441883174308C30A84000008FE
:100050000800483465346C346C346F3420345734C1
:0A0060006F3472346C3464340034E1
:1009D00083010800F0000030711870070310F00D5B
:1009E0000310F10CF10803190800EC2CF401F501D7
:1009F0000310F30CF20C031C042D7008F4077108AB
:100A00000318710AF5070310F00DF10D7208730455
:100A100003190034F82C8301B50083161114111842
:100A20000F2D83128C11C63093008C1D152D8C1147
:100A300093018C1D192D8C113508840083138008B7
:100A400003192A2D3508840000089300B50A8C1973
:100A50001B2D272D8316111511192C2D831208001B
:100A60008301B500831611141118342D83128C11D3
:100A7000C63093008C1D3A2D8C1193018C1D3E2D98
:100A80008C11023093008C1D432D8C11350893007E
:100A90008C1D482D8C118316111511194D2D8312A3
:100AA00008008316031311141118542D83128C118E
:100AB000C63093008C1D5A2D8C1193018C1D5E2D18
:100AC0008C110C3093008C1D632D8C11043093001D
:100AD0008C1D682D8C118316111511196D2D831223
:100AE000080083160313860183128601FF308316E4
:100AF0008700831287008030831694003830831279
:100B00009400831691010A30930001308312900003
:100B100081309F00803083169F008312B501B6019B
:100B2000B701B801B50A0319B60A0319B70A0319C0
:100B3000B80A00303802031DA72D00303702031D0C
:100B4000A72DEA303602031DA72D603035020318A9
:100B50000800922D712551251A3030252930B60014
:100B60000030B70020300A128A11BB250A128A1100
:100B700020300B25BA2D8301BE00BC013508B90019
:100B8000AE2F3D08253A031D9F2FFF30BA00BB0151
:100B9000B801612FBE080319D12D3E0884008313CC
:100BA00080013C0808000230B90739028400831331
:100BB00000089D2FB80AE02D0830BA07FE30BA07AA
:100BC0000230B9073902840083130008BF00840A89
:100BD0000008C0003818C01FF42DBF09C009BF0AA3
:100BE0000319C00ABB03F52DB8010B30BA073A0848
:100BF000F200F3014008F1003F08F0000A128A11E8
:100C0000C6277008BD003A08F200F3013F08F00063
:100C10004008F1000A128A11C6270A128A117408C4
:100C2000BF007508C000C101C10AC20142084002EC
:100C3000031D1C2E41083F02031C412E3A08F200FE
:100C4000F3014108F0004208F1000A128A11F6246B
:100C50000A128A117408C1007508C200BB03162E5F
:100C6000BC0ABE0803193B2E3E08840083132030C3
:100C70008000BE0A412E20300A128A11E8240A128E
:100C80008A11BB033B08803A7F3E0318302E381C84
:100C9000562EBC0ABE080319522E3E088400831348
:100CA0002D30912E2D300A128A11E8243A08F200D4
:100CB000F3014108F0004208F1000A128A11C62728
:100CC0000A128A117408C1007508C2004104031990
:100CD000972E4208F3004108F2004008F1003F0857
:100CE000F0000A128A11C6277408F0007508F10096
:100CF0003A08F200F3010A128A11C6270A128A1171
:100D00007008BB00803A763E031C882E0730BB0774
:100D1000BC0ABE080319942E3E08840083133B08C6
:100D2000303E8000BE0A562E3B08303E532E0A301D
:100D30003D02031C9D2E0730BD07BC0ABE080319E7
:100D4000A72E3E08840083133D08303EA72F3D08A0
:100D5000303EAB2FBC0ABE080319B52E3E088400F6
:100D6000831320308000BE0ABB2E20300A128A1165
:100D7000E8240A128A11BB033B08803A7E3E03181E
:100D8000AA2E0230B9073902840083130008BD007F
:100D90009F2F0230B9073902840083130008C10075
:100DA000840A0008C200BD013D084107C300420893
:100DB000C40043080318C40A0A128A1113200A1235
:100DC0008A1100380319E62EBD0AD42E3A083D02D6
:100DD0000318EC2E3D08BA003A08BB1B232FFF3A3C
:100DE0003B07031C232FBC0ABE080319FE2E3E0836
:100DF0008400831320308000BE0A042F20300A12A2
:100E00008A11E8240A128A11BB03EC2E4208C4009E
:100E100041080A128A1113200A128A11BD00C10A60
:100E20000319C20ABC0ABE0803191D2F3E0884001C
:100E300083133D088000BE0A232F3D080A128A1141
:100E4000E8240A128A11BA033A0F062FAE2F370888
:100E5000C40036080A128A1113200A128A112A3A8B
:100E6000031D392F0230B9073902840083130008AB
:100E70005D2F3708C40036080A128A111320D03EAD
:100E8000BA00B60A0319B70A3708C40036080A12AE
:100E90008A1113200A128A11BD0030303D02031C52
:100EA000612F3A303D020318612F0A30F1003A08F1
:100EB0000A128A11EA243D07D03EBA00B60A031985
:100EC000B70A3708C4003608B60A0319B70A0A1267
:100ED0008A1113200A128A11BD00003A0319CA2D83
:100EE0002A3A0319D32D043A0319272F763A031906
:100EF000DC2D3B3A0319BC2E073A0319DA2D0B3AC5
:100F00000319DE2D1C3A0319C92E063A0319E02DE8
:100F10000D3A0319DC2D30303D02031C9F2F3A306F
:100F20003D0203189F2F0A30F1003B080A128A1174
:100F3000EA240A128A113D07D03EBB00612FBC0A89
:100F4000BE080319AA2F3E08840083133D088000C1
:100F5000BE0AAE2F3D080A128A11E8243708C400E1
:100F60003608B60A0319B70A0A128A1113200A12A0
:100F70008A11BD00BD08031DC12DBE080319C42F71
:100F80003E088400831380013C080800F601F40148
:100F9000F50172087304031DD02FF001F101003434
:100FA0001F30F6040310F60AF20DF30D031CD32FC5
:100FB000F30CF20C73087102031DE02F720870022B
:100FC000031CE82F7208F0027308031C730AF10275
:100FD000F40DF50DF60BF61AD82FF61FF42FF409C1
:100FE000F40A0319F503F5097408F2007508F30013
:100FF000761F0034F009F00A0319F103F1090034F7
:02400E00323B43
:00000001FF
